:100000000C943B060C9463060C9463060C94F70E58
:100010000C9463060C94C80E0C9463060C9463064F
:100020000C9463060C9463060C9463060C94250CE4
:100030000C9463060C9463060C9463060C9463069C
:100040000C940A0E0C9463060C949C0E0C9463069C
:100050000C9463060C94250F0C9463060C946306B1
:100060000C9463060C94630604156C15DC15451698
:10007000A016A016A0161C171C1706180618F718AD
:100080005D19C1192A1A272143217F21BA21F5219F
:10009000FA21122254226E225A215F2155215A211F
:1000A0005F215A215F2107634236B79BD8A71A39CF
:1000B000685618AEBAAB558C1D3CB7CC5763BD6DB6
:1000C000EDFD753EF6177231BF000000803F05A8B8
:1000D0004CCDB2D44EB93836A9020C50B9918688AD
:1000E000083CA6AAAA2ABE000000803F0664EC1BBA
:1000F0003C04BC163E3BE5B93CC93C37C29E5A3D68
:10010000660498083EEA69AAAA3E000000803F0003
:10011000000C1925313C47515A626A70757A7D7E10
:100120007F7E7D7A75706A625A51473C3125190C81
:1001300000F4E7DBCFC4B9AFA69E96908B8683828E
:10014000818283868B90969EA6AFB9C4CFDBE7F4FD
:10015000000810182028303840474F575F676F77E6
:100160007F776F675F574F47403830282018100857
:1001700000F8F0E8E0D8D0C8C0B9B1A9A199918938
:1001800081899199A1A9B1B9C0C8D0D8E0E8F0F8A7
:100190007F7B77736F6B67635F5B57534F4B47434F
:1001A000403C3834302C2824201C1814100C08042F
:1001B00000FCF8F4F0ECE8E4E0DCD8D4D0CCC8C41F
:1001C000C0BDB9B5B1ADA9A5A19D9995918D898500
:1001D00081818181818282828282828383838384FE
:1001E000848485858686878788898A8A8B8C8D8F8B
:1001F0009091939597999B9DA0A3A6A9ADB1B6BBED
:10020000C0C6CCD3DBE3ECF5000C18263545576BA4
:1002100000193046586670767876726C655F59566C
:100220005556595F656C7276787670665846301907
:1002300000E7D0BAA89A908A888A8E949BA1A7AA30
:10024000ABAAA7A19B948E8A888A909AA8BAD0E775
:100250007F7F7F7F81818181818181818181818196
:10026000818181818181818181818181818181817E
:10027000818181818181818181818181818181816E
:10028000818181818181818181818181818181815E
:100290007F7F7F7F7F7F7F7F7F7F7F7F7F7F7F7F6E
:1002A000818181818181818181818181818181813E
:1002B000818181818181818181818181818181812E
:1002C000818181818181818181818181818181811E
:1002D0007F7F7F7F7F7F7F7F7F7F7F7F7F7F7F7F2E
:1002E0007F7F7F7F7F7F7F7F7F7F7F7F7F7F7F7F1E
:1002F00081818181818181818181818181818181EE
:1003000081818181818181818181818181818181DD
:100310007F7F7F7F7F7F7F7F7F7F7F7F7F7F7F7FED
:100320007F7F7F7F7F7F7F7F7F7F7F7F7F7F7F7FDD
:100330007F7F7F7F7F7F7F7F7F7F7F7F7F7F7F7FCD
:10034000818181818181818181818181818181819D
:100350007F7F7F7F7F7F7F7F7F7F7F7F7F7F7F7FAD
:100360007F7F7F7F7F7F7F7F7F7F7F7F7F7F7F7F9D
:100370007F7F7F7F7F7F7F7F7F7F7F7F7F7F7F7F8D
:100380007F7F7F7F7F7F7F7F7F7F7F7F8181818175
:100390000004080C1014181C2024282C3034383C7D
:1003A0004043474B4F53575B5F63676B6F73777B7C
:1003B0007F7F7F7F7F7F7F7F7F7F7F7F7F7F7F7F4D
:1003C0007F7F7F7F7F7F7F7F7F7F7F7F7F7F7F7F3D
:1003D0007F7F7F7F7F7F7F7F7F7F7F7F7F7F7F7F2D
:1003E0007F7F7F7F7F7F7F7F7F7F7F7F7F7F7F7F1D
:1003F0007F7B77736F6B67635F5B57534F4B4743ED
:10040000403C3834302C2824201C1814100C0804CC
:100410007F7F7F7F7F7F7F7F7F7F7F7F7F7F7F7FEC
:1004200081818181818181818181818181818181BC
:100430007F7F7F7F7F7F7F7F8181818181818181BC
:100440007F7F7F7F7F7F7F7F8181818181818181AC
:100450007F7F7F7F7F7F7F7F81818181818181819C
:100460007F7F7F7F7F7F7F7F81818181818181818C
:100470007F7F7F7F7F7F7F7F7F7F7F7F7F7F7F7F8C
:100480007F7F7F7F7F7F7F7F81818181818181816C
:1004900098B8F25BDD26ECEB532F16B79198E41B6E
:1004A0004F192290D31424E284B6A1383FA55E4EA2
:1004B00087E53192E718F70BB041F6C89B74693AAB
:1004C000BD94815FB95836FE536DDB3B28B354E4CD
:1004D0007F7F7F7F7F7F7F7F7F7F7F7F7F7F7F7F2C
:1004E0007F7F7F7F7F7F7F7F7F7F7F7F7F7F7F7F1C
:1004F0007F7F7F7F7F7F7F7F7F7F7F7F7F7F7F7F0C
:100500007F7F7F7F7F7F7F7F7F7F7F7F7F7F7F7FFB
:1005100000000000000000000000000000000000DB
:100520002B2724271F1B181B130F0C0F0703000377
:10053000003C043909340C30102D152818241C2DCA
:1005400010401F001F40100010401F001F4010806F
:100550001505020507050400150502050705040039
:10056000020502050407040700040004090109014B
:1005700000408007408003408005408002800202E6
:100580000C21130E0C150702020407150E1013217F
:1005900000800303058007070880161617170F4011
:1005A00000400780004007048004078000048004A6
:1005B0000003070A0C0F1316181B1F2224272B2ECB
:1005C00000400C400B4007400C4040800B4007406F
:1005D00029241D18110C050027241D18110C0500D5
:1005E0000040050700000507004005070005070C4F
:1005F000000C0007000A000700090007000A0007B6
:1006000018171A151A1318121810180E180C180BA0
:1006100080808080808080808080808080808080DA
:100620007F7F7F7F7F7F7F7F7F7F7F7F7F7F7F7FDA
:100630004B595C5C5C5B5A59F5EBE8E7E61C51559D
:10064000FEF2F0EFEFEFEFEF8982808081BBF0F6F2
:10065000737E51FE8697A6BD525D686DF09C8095B5
:100660002E3A464DCFDEECF90714212BACBBCADB8A
:100670006A7F7D7C7B7A7979DCD1D2D2D2D3D3D315
:10068000D4D4D5D5D5D6D6D6D7D7D7D8D8D8D9DDFE
:1006900080878F979FA7AFB7BFC7CFD7DFE7EFF7A9
:1006A000FF070F171F272F373F474F575F676F779A
:1006B00007141F2C37434E59646E777F45A6E10817
:1006C000DFA7C3D8D2CE93AFBDC0C6D0DCE6F0FB67
:1006D000808594A7BBD0E4F90E2216E6F7091D2FFA
:1006E000E3F1021629FBEAFB0F22364A5D63212D56
:1006F00040515D666F777E7904060C141D263033F9
:10070000C6CAD1DBE5EFFA00808188909AA4AFC019
:10071000E6C3A49286808B89AAA4D6C600E81A00F4
:1007200015191A1F39325C4A755B7A59633F300AD2
:10073000FF172F465969757C7F7C756959462F17BD
:10074000FFE7CFB8A595898280828995A5B8CFE7C4
:10075000122F2C446D6C62797F6A5E6A5328221DC9
:10076000E7D3D5B491989A8181999A91B1D6D6E47C
:100770002C393E42484F5A787E55453A312A241C3E
:10078000CFC4C0BBB6AEA38680A8B9C4CCD3DAE2CE
:10079000800707060605050404030303020202019D
:1007A0000101010000000000FFFFFFFFFFFFFE014D
:1007B000CADC7F639B851E6B0DB2D52B2EEFD5FB5C
:1007C0001D0CEDEE060EFFF4FA0605FCF9FF040120
:1007D0001B1E190F100A0B080B050803050106FF65
:1007E00002FE03FE01FDFFFE02FE01FD00ED80CCD6
:1007F00000000000000000000000000000000000F9
:1008000000000000000000000000000000000000E8
:100810009CBF0A07DFC4DB01EAACD3F6EDEFCB19CE
:10082000250D3C40F1417F220909F5D41F2A3102F0
:100830005D23C68005181E4B2CB8D93BF90D0A2242
:10084000DD424D34C90715E1BEC9D5980707FEFA48
:100850000C251919647178DCC57F736324081209AB
:10086000F1DAD1DCCC8C8482273A8999ADF208F296
:1008700077F01A3242B9CC033E0F06DF6A057D6677
:100880009980F79320F7EFC2FC3045BFCEE4108E7D
:1008900025CF1FC214E480465613C05E0459DE2FD4
:1008A0000F8E60F0EFBD4137BA1AB43DC7E80AB306
:1008B0002C777E6F3507F9020B00E7CCBDC4D8F169
:1008C0000F283B403015FBF1FB04F5C68D808AD51F
:1008D000808CB18C8E8087CA12F5F1121D10060330
:1008E000FBFAEDE3F11406F046757F6D684E716E0C
:1008F0001C24262625242123432C1D16110E0D0D04
:1009000029170C06030100F680899CADBDCCD9E8FF
:100910008081899ACCD50A160A1C3211F5E5F419A2
:10092000E50B1908ECCCE4F5E9F62B3365737A7F17
:10093000235E7647335458401B1306BE919280A223
:10094000ED3057403E37C9A0CAF90DDBBAC3B6D85F
:10095000457E7D7851F8A2808FB6E30F3A627969BF
:1009600020C08780839C10767E5AA941ED8385C084
:100970008018891B921D9A1EA317AC16B416BD10C1
:10098000D817F11E0725192C2B2F36363F3D453839
:100990002823CEE02B008BDDEA340B08180FE11082
:1009A0005F5E80BAF61CE6EFF8E4D0213371DCE13B
:1009B000E3D974E29F65F6E9C858F08068FDE1CD9F
:1009C0004D248D5921D1CA4221910549D0B95905EB
:1009D0006878781D808B931E764A57B8B6CAC23F96
:1009E000044715FC1FA7E3B8F9664B6FC79985A5A7
:1009F0001C5630CBB0EC263DEE20B8F42EDAF9329E
:100A0000FEFFDECB07404BE699D611497F9FA3E05E
:100A1000000101020203040405050607070809098D
:100A20000A0B0B0C0D0D0E0F0F10111212131414D4
:100A30001516171718191A1B1B1C1D1E1F1F202106
:100A40002223242525262728292A2B2C2D2E2F2F1B
:100A5000303132333435363738393A3B3D3E3F401A
:100A600041424344454648494A4B4C4D4F505152F0
:100A700053555657595A5B5C5E5F606263646667A4
:100A8000696A6B6D6E707173747677797A7C7D7F2D
:100A9000210023002500270029002C002E00310012
:100AA000340037003A003E004100450049004E0046
:100AB000520057005C00620068006E0075007B0009
:100AC00083008B0093009C00A500AF00B900C40018
:100AD000D000DC00E900F70006011501260137010E
:100AE0004A015D01720188019F01B801D201EE0146
:100AF0000B022A024B026E029302BA02E4021003B6
:100B00003F037003A403DC03170455049704DD04BA
:100B100027057505C80520067D06E0064907B807C4
:100B20002D08A9082D09B9094D0AEA0A900B400CB5
:100B3000FA0CC00D910E6F0F5A1053115B12721305
:100B40009A14D41520178018F519801B231DDE1E5A
:100B5000B420A622B524E4263429A72B402E003148
:100B6000EA330037453ABC3D68414C456B49C84DB6
:100B700068524F57805C0062D467006E8A74797B3C
:100B8000D082978AD592909BD0A49DAEFFB8FFC328
:100B90000605041005030F040210010F000E0000EB
:100BA0000100010001005515030001005515030067
:100BB000010055550100555501005555020004002E
:100BC000000005000E001B002E004D007B00C3003E
:100BD0003201DD01E4027904E806A80A6F10541915
:100BE00000000008001100190022002A0033003B19
:100BF0000044004C0055005D0066006E0077FF7FEA
:100C00000F00000F0007000F0000000000070700A2
:100C10000003050507070B0B000507000307070F77
:100C2000FF7FFF0F9005AA027401D90085005600CE
:100C3000390026001A0013000D0009000700050006
:100C400000000000000000000303050707070B0F6A
:100C50000004090102030B0E00010407080C0D0F2C
:100C6000000000000000000001010101010101007D
:100C70000FF09222912211241FBECFEFD8E0DEBFE9
:100C8000CDBF11E0A0E0B1E0E8EDFAE502C00590CB
:100C90000D92AA36B107D9F723E0AAE6B1E001C068
:100CA0001D92AA3DB207E1F716E0CAE3D6E004C000
:100CB0002197FE010E94272CC933D107C9F70E9452
:100CC000C00F0C945F2D0C940000089508950895B2
:100CD00008950895462FDC011496ED91FC91159727
:100CE0000088F189E02D683F48F16C3F28F46A3FA5
:100CF00060F4683F21F008956C3FB1F0089581855C
:100D000092850196928781870895128611861486AE
:100D1000138681E0848382819381DC01ED91FC91D3
:100D20000480F581E02D09C0148282819381DC0169
:100D3000ED91FC910680F781E02D0994603F70F100
:100D40001092D601603FA9F481E0858316828FEF6F
:100D500080930601809305018085882309F4EEC005
:100D600082819381DC01ED91FC910084F185E02D7D
:100D7000E4CF673F09F0E2C08581882309F4DEC033
:100D800015828085882309F4D9C082819381DC0192
:100D9000ED91FC910484F585E02DCFCF67FF0BC06A
:100DA0006093D60181E08093D5011092D401109216
:100DB000D301158208958581882331F1668181E010
:100DC000860F8683813019F440930601089582309E
:100DD00019F44093050108959091060180819813BC
:100DE000ADC09091050187819813A8C080858823A4
:100DF00009F4A4C082819381DC01ED91FC916250E1
:100E00000284F385E02D09948091D601882309F4AA
:100E100095C09091D5019923C1F06093D4011092AF
:100E2000D501DF01A257BF4F9C91992309F486C0D9
:100E30009181906C891382C082819381DC01ED9154
:100E4000FC910488F589E02D09946093D301918188
:100E5000292F206982131BC06623C9F06091D40139
:100E6000DF01A60FB11D1E968C911E9781115FC0E8
:100E700081E01E968C9385858F5F85878281938123
:100E8000DC01ED91FC910190F081E02D2EC0392F15
:100E90003068831721F082131AC0411118C0609185
:100EA000D401DF01A60FB11D1E968C911E978823D9
:100EB000F1F11E961C9285858150858782819381F0
:100EC000DC01ED91FC910280F381E02D2FC0292FF0
:100ED000206B82130CC082819381DC01ED91FC9127
:100EE0000088F189E02D6091D401099520C0906EB1
:100EF00089131DC082819381DC01ED91FC91411128
:100F000005C00288F389E02D61E810C04F3729F44D
:100F10000288F389E02D6FE709C0642F70E0605408
:100F20007109660F771F0288F389E02D09951092E9
:100F3000D4011092D30181E08093D50108950895E2
:100F400008950895CF93DF93EC01FC01EB5BFE4F16
:100F500060838AE0689F90011124245C3F4F40E049
:100F600050E060E078E98AE390E00E94E4272A8775
:100F70003B874C875D87AE85BF850E94D127AA2716
:100F8000BB278E839F83A887B987DF91CF91089570
:100F9000CF93DF93EC01E62FF0E0EE0FFF1FE05759
:100FA000F54F85919491FE01E357FF4F20813181E8
:100FB0008217930771F0248135818217930749F0D6
:100FC000918380833383228314861386CF010E940A
:100FD0006D0E81E088A789A78FA1882311F01DA23B
:100FE0001CA281E08EAB8FAB8DA9882311F01BAAC8
:100FF0001AAADF91CF910895DC0157966C93579709
:1010000058968D919C915997DC01ED91FC9102804D
:10101000F381E02D09940F931F93CF938C01C0E0CF
:10102000D80112968D919C911397DC01ED91FC9162
:101030000280F381E02D6C2F0995CF5FC03881F7D6
:10104000CF911F910F9108958F929F92AF92BF926F
:10105000CF92DF92EF92FF92CF93DF93EC018881E2
:101060009981AA81BB81860F911DA11DB11D888325
:101070009983AA83BB83CC80DD80EE80FF808C15B2
:101080009D05AE05BF0540F08C199D09AE09BF094D
:1010900088839983AA83BB8388819981AA81BB8134
:1010A000009720E1A207B105A8F4009728E0A20765
:1010B000B10590F4009724E0A207B10578F40097F9
:1010C00022E0A207B10560F4009721E0A207B10574
:1010D00018F008C035E007C034E005C033E003C0B5
:1010E00032E001C031E040E150E0431B5109BC0156
:1010F000CD0104C0660F771F881F991F4A95D2F74C
:101100004601570104C0B694A794979487943A95E2
:10111000D2F7A50194010E94E42739872887DF913F
:10112000CF91FF90EF90DF90CF90BF90AF909F90C6
:101130008F900895CF92DF92EF92FF920F931F93BB
:10114000FC018585882309F46FC08485823071F1A4
:1011500030F4882309F45FC0813041F065C08330EA
:1011600009F441C0843009F443C05EC0208131815C
:10117000A62FB0E00E94062840855185AFEFBFE75B
:101180008D01041B150B012E000C220B330B601775
:1011900071078207930728F082E08487B187A087D0
:1011A00043C0640F751F718760873EC02281338101
:1011B000A62FB0E00E94062820853185A481B58144
:1011C000A9014A1B5B0B6A01550FEE08FF086C155D
:1011D0007D058E059F0528F083E08487B187A08771
:1011E0001CC0C9011DC0848195819187808715C06D
:1011F00026813781A62FB0E00E94062840855185C0
:101200008A01052E000C220B330B60177107820731
:10121000930728F0148611861086158605C0CA012A
:10122000861B970B918780871F910F91FF90EF90FE
:10123000DF90CF900895DC011C968C911C97199635
:101240002C911997813099F4822F922F990F990B35
:1012500097FF03C0919581959109EFE7F0E0E81BB6
:10126000F109E05FF54F9491EFE7E91B0DC0E22F24
:10127000F22FFF0FFF0BF7FF03C0F195E195F10986
:10128000FF27E05FF54FE4911A968C91882319F0BF
:101290008E2F819508958E2F0895CF92DF92EF9231
:1012A000FF92CF936A017B01C22F682F880F770BC3
:1012B000880B990B0E946B2920E030E04EEF52E43E
:1012C0000E948728A70196010E94D32A0E94012923
:1012D0006B017C016C2F70E080E090E00E94692936
:1012E0009B01AC01C701B6010E94D32A20E030E087
:1012F00040E85FE30E9415280E94402B0E943A2993
:10130000862FCF91FF90EF90DF90CF900895FC0152
:1013100036E0639FE00DF11D1124E40FF11D2287DB
:10132000DC0156968D919C915797009739F0DC011E
:10133000ED91FC910480F581E02D09940895242F0E
:10134000DC011496ED91FC911597462F67898289EF
:1013500093890C948709DC01262F2170E22FF0E09D
:10136000E059F34F849170E075956795A60FB71F0C
:101370009C91892390E0220F220F02C095958795BA
:101380002A95E2F708950F931F93CF93DF93EC0113
:101390006E8BE88DF98D0190F081E02D0081118137
:1013A0008A899B890E94AB0920E0482F6E89888D2D
:1013B000998DF801DF91CF911F910F910994CF93EF
:1013C000DF93EC01A62FB0E0B595A795962F91700D
:1013D000E92FF0E0E059F34FE491AC0FBD1F2E2F41
:1013E00020958C918223990F990F242F01C0220FF1
:1013F0009A95EAF7E223E82BEC938E899F89009770
:1014000049F0DC01ED91FC910190F081E02DDF913C
:10141000CF910994DF91CF910895CF93DF93EC01A1
:1014200040E060E08A899B890E94DF0941E061E039
:101430008A899B890E94DF0941E062E08A899B8951
:101440000E94DF0942E063E08A899B890E94DF09EC
:1014500040E064E08A899B890E94DF0945E065E0FD
:101460008A899B890E94DF0940E066E08A899B891E
:101470000E94DF0941E067E08A899B890E94DF09B9
:1014800046E068E08A899B890E94DF092FEF41E0EE
:1014900060E08A899B890E9487092FEF42E060E023
:1014A0008A899B890E94870920E043E060E08A895D
:1014B0009B890E94870920E044E060E08A899B893B
:1014C0000E94870920E045E060E08A899B890E94AC
:1014D00087092FEF40E060E08A899B890E94870995
:1014E0002CE841E061E08A899B890E94870920E01D
:1014F00042E061E08A899B890E94870920E043E0FD
:1015000061E08A899B890E94870920E044E061E0CC
:101510008A899B890E94870920E045E061E08A89E9
:101520009B890E9487092CE340E061E08A899B89BE
:10153000DF91CF910C948709CF92DF92FF920F93A6
:101540001F93CF93DF93CDB7DEB767970FB6F894AD
:10155000DEBF0FBECDBFDC011696ED91FC91179753
:10156000DF01A856BF4FFC90613009F06BC08C01C1
:101570002F2D20952770EC59FF4F3081FC0184817D
:101580009581313081F42F8B0E940D0AD801169677
:101590008D919C9117972F894F2D62E088569F4F10
:1015A0000E94830F4FC0DC015296ED91FC9153973E
:1015B000AF01CE0101966C0138E0380FDA016D9170
:1015C000AD01D6016D936D013A13F8CFAF01465FBF
:1015D0005F4FBE01675F7F4F6F01B0E1CB0ED11C43
:1015E000DA013D91AD01DB013D93BD014C155D0577
:1015F000B9F7AE01415F5F4FBF016A5E7F4FD60111
:101600003D916D01DA013D93AD01C616D706B9F7DC
:1016100030853D8B31853E8B46E150E060E070E0E7
:101620002F8B0E949027F801868197812F894F2D5B
:1016300064E088569F4F0E94830F6FE78FEF93E01F
:101640000E94A02767960FB6F894DEBF0FBECDBFED
:10165000DF91CF911F910F91FF90DF90CF90089570
:101660000F931F93CF93FC0184819581DC015696E3
:10167000CC91413009F070C0613059F4C11102C001
:1016800067E002C06FEF6C0FCF911F910F910C9428
:10169000C3098F01623049F4C73011F460E002C021
:1016A00061E06C0F0E94C3097AC0633041F5068087
:1016B000F781E02DEC59FF4F2081FC01828993894D
:1016C000213041F468E00E94AB09882309F467C027
:1016D0004FEF28C06C2F0E94AB09D8011496ED91F2
:1016E000FC911597811109C04FE06C2F8289938975
:1016F000CF911F910F910C94DF094FEF2BC06430F5
:10170000E9F50680F781E02DEC59FF4F208121306B
:1017100089F468E0FC01828993890E94AB098F30CB
:10172000F0F541E0480FD8011496ED91FC91159722
:1017300068E0DCCF6C2FFC01828993890E94AB09A1
:10174000D8011496ED91FC9115978F3011F440E07B
:10175000CCCF41E0480FC9CF611108C0FC0180899E
:101760009189CF911F910F910C940B086530B9F4BA
:10177000642FCF911F910F910C94FC076111F6CF4C
:10178000DC01ED91FC911197AD53BF4F0190F081B9
:10179000E02D4FE76C91CF911F910F910994CF915C
:1017A0001F910F910895CF92DF92EF92FF920F93C6
:1017B0001F93CF93DF93CDB7DEB78C01EDB6FEB6A6
:1017C000DC014C9114968D919C911597FC01649FBE
:1017D000E00DF11D1124BF0150E02DB73EB7241BD1
:1017E000350B0FB6F8943EBF0FBE2DBF8DB79EB719
:1017F00001966C010E94782790E0F801808198178B
:10180000B0F4292F30E0F601E20FF31F8081D801F8
:101810001696ED91FC911797418152814115510522
:1018200021F0FA01E20FF31F80839F5FE6CF0FB62E
:10183000F894FEBE0FBEEDBEDF91CF911F910F91C8
:10184000FF90EF90DF90CF9008951F920F920FB608
:101850000F9211242F933F934F936F937F938F9306
:101860009F93AF93BF93EF93FF9380916E01882373
:1018700049F0609102018091D2010E941B2C9923B2
:1018800009F45AC03091D20131110FC080916F011B
:10189000882331F081E08093730110926F0105C0BD
:1018A0008091730181111092730180917301E09115
:1018B000D001F091D1018823D1F0A0917101B091B4
:1018C000720111968D919C911297009721F0DC0185
:1018D000A30FB11D2C9181819281009721F0FC0111
:1018E000E30FF11D208320582093B4000BC08181A9
:1018F0009281009721F0FC01E30FF11D40814058D7
:101900004093B40090910301209104018091D20191
:10191000820F89238093D201FF91EF91BF91AF9104
:101920009F918F917F916F914F913F912F910F9048
:101930000FBE0F901F9018958091000190910101AA
:101940009093890080938800809102018093040124
:1019500010926E0197CFFC01EE53FF4F6083089504
:10196000FC0116821782108611861786168680E083
:1019700096E0A0E0B0E082879387A487B587EC5417
:10198000FF4F0190F081E02D80E1878380E881871F
:101990000895CF93DF93FC01DC01A60FB11DAD01CB
:1019A0004B535F4FDA018C918823F9F0EF01C0545B
:1019B000DF4F88819F012F533F4FD9018C93815076
:1019C0008883DA011C92811110C0DF01AC54BF4F33
:1019D0000D90BC91A02D12968C91811106C094E0BF
:1019E00090A781E081A796AB87ABDF91CF91089557
:1019F0000E945A2DCF93DF93EC011E821F8218861E
:101A000019861F861E86FC01EB5BFE4F60810E94DB
:101A1000A207CC54DF4FE881F98180E1878380E819
:101A20008187DF91CF910895CF93DF93FC01E60F7B
:101A3000F11DEB53FF4F208121111DC0DC01A0548B
:101A4000BF4F2C91EC01CF53DF4F28832F5F2C9396
:101A500021E02083FC01EC54FF4F0190F081E02D48
:101A60002281211104C0DF91CF910C94C807FC01A1
:101A7000EC53FF4F6083DF91CF910895FC016734F1
:101A800009F497C028F5613109F460C078F4653035
:101A900009F448C020F4613009F43FC0089567306C
:101AA00009F448C0603109F44DC00895623209F468
:101AB00064C038F4603209F44DC0613209F455C095
:101AC0000895633209F461C0643209F466C0089570
:101AD0006B3509F486C078F46D3409F476C020F4CF
:101AE0006A3409F462C008956E3409F466C06F3434
:101AF00009F46FC008956E3509F47FC038F46C3571
:101B000009F473C06D3509F474C008956F3509F494
:101B100078C06B3709F47AC0089550E09A01359582
:101B2000279555C050E0B3E055954795BA95E1F734
:101B300066E017C0242F220F40E060E0828993897D
:101B40000C948709242F220F42E0F7CF242F220F75
:101B500045E0F3CF50E0A3E055954795AA95E1F70E
:101B600060E0828993890C94DF0950E073E0559519
:101B700047957A95E1F761E0F4CF50E063E0559541
:101B800047956A95E1F762E0ECCF50E033E0559578
:101B900047953A95E1F763E0E4CF50E023E05595AF
:101BA00047952A95E1F767E0DCCF242F220F41E02B
:101BB000C4CF242F220F41E027C050E093E0559579
:101BC00047959A95E1F764E0CCCF242F220F43E0AC
:101BD0001BC050E083E0559547958A95E1F765E095
:101BE000C0CF242F220F44E00FC0242F220F44E047
:101BF000A4CF242F220F43E0A0CF242F220F42E0B6
:101C000003C0242F220F45E061E098CF808991899D
:101C10000C940B081F920F920FB60F9211242F9362
:101C20003F938F939F93AF93BF9380916A0190915D
:101C30006B01A0916C01B0916D013091DC0123E04A
:101C4000230F2D3720F40196A11DB11D05C026E8F4
:101C5000230F0296A11DB11D2093DC0180936A0120
:101C600090936B01A0936C01B0936D018091D801AA
:101C70009091D901A091DA01B091DB010196A11DEB
:101C8000B11D8093D8019093D901A093DA01B0934C
:101C9000DB01BF91AF919F918F913F912F910F9059
:101CA0000FBE0F901F901895FC01808191810097C5
:101CB00011F00C94C22C0895FC011182108216823E
:101CC0001086178211861286138684E18487158612
:101CD00064836583538342830895CF93DF93EC013C
:101CE000AF81B885109719F41A86198622C08E81A3
:101CF0008823E9F0488159818A819B81EC81FD81AB
:101D00008417950738F49A012E1B3F0B0E94062872
:101D10009F0106C09F01241B350B0E9406289A01D3
:101D200040E050E00E94E4273A87298702C0BA8742
:101D3000A987DF91CF9108951F920F920FB60F924E
:101D400011242F938F939F93EF93FF938091C00063
:101D50009091C6008091C1018F5F8F732091C20165
:101D6000821304C084E08093800108C0E091C10127
:101D7000F0E0EF57FE4F90838093C101FF91EF9108
:101D80009F918F912F910F900FBE0F901F901895DC
:101D90001F920F920FB60F9211242F934F935F93C0
:101DA0008F939F93EF93FF9329B1822F90E0AC0123
:101DB00055954795559547954170E4E7F1E0408387
:101DC000221F2227221F248324E0959587952A9598
:101DD000E1F781708583FF91EF919F918F915F91E2
:101DE0004F912F910F900FBE0F901F9018951F923B
:101DF0000F920FB60F9211242F934F935F938F93EF
:101E00009F93EF93FF9323B1822F90E0AC01E5E025
:101E100055954795EA95E1F74170E4E7F1E0418394
:101E200044E0959587954A95E1F78170828321700A
:101E30002383FF91EF919F918F915F914F912F910C
:101E40000F900FBE0F901F9018951F920F920FB614
:101E50000F9211248F93EF93FF93E091D701F0E05D
:101E600080917900E658FE4F80838091D7018F5F83
:101E70008093D7018091D701863010F01092D7015E
:101E80008091D70180937C0080917C008064809356
:101E90007C0080917C00806280937C008FE880933E
:101EA0007A0080917A00806480937A00FF91EF91AC
:101EB0008F910F900FBE0F901F901895FC01E85660
:101EC000FF4F208121FF02C0299A01C0299820815B
:101ED00022FF02C02B9A01C02B98208120FF02C054
:101EE0002A9A01C02A98FC01E356FF4F808181FFA6
:101EF00002C05D9A01C05D98808180FF02C05E9A39
:101F000008955E980895CF93DF93DC0112966C9349
:101F1000129714961C921497C1E7DCE0FE0194918D
:101F200060E77CE0FB018491592F509513963C911A
:101F3000139735239078932B382F309593238870FF
:101F4000892B13968C931397FE01C491FB01649126
:101F50003C2F309511968C9111973823F0E14F9FCB
:101F6000C00111248C23832B962F9095892326233F
:101F7000282B11962C9311974C93DF91CF910895B4
:101F8000CF93DF93CDB7DEB7C654D1090FB6F8941F
:101F9000DEBF0FBECDBF789484B5826084BD84B5AA
:101FA000816084BD85B5826085BD85B5816085BD54
:101FB00080916E00816080936E001092810080910C
:101FC0008100826080938100809181008160809394
:101FD0008100809180008160809380008091B100B9
:101FE00084608093B1008091B00081608093B000E4
:101FF00080917A00846080937A0080917A00826078
:1020000080937A0080917A00816080937A00809139
:102010007A00806880937A001092C1008091C0009D
:1020200082608093C0001092C5008FE38093C4004B
:102030008091C10080618093C1008091C10088605F
:102040008093C1008091C10080688093C10080911D
:10205000C1008F7D8093C1008091C9019091CA0118
:10206000FC01E856FF4F21E02083359620830E9433
:102070005E0FC090C701D090C8018091B6008F7BE1
:102080008093B6008091B6008F7D8093B6008091DA
:10209000B00081608093B0008091B0008260809336
:1020A000B0008091B100877F8093B1008091B00033
:1020B0008F7E8093B0008091B00080628093B000EA
:1020C0008091B0008F7B8093B0008091B0008F77BB
:1020D0008093B0008091B10081608093B1008091C5
:1020E000B1008D7F8093B1008091B1008B7F809390
:1020F000B100F894809180008E7F80938000809161
:1021000080008D7F80938000809181008860809323
:102110008100809181008F7E809381008091810079
:10212000816080938100809181008D7F8093810008
:10213000809181008B7F809381008091000190913C
:102140000101909389008093880080916F008260E4
:1021500080936F007894D6015096ED91FC91519741
:10216000118252960D911C91539746E150E060E028
:1021700070E0CE0101960E947827FE0131963F0162
:10218000512C30E7832E3CE0932E41E7A42E4CE007
:10219000B42E7301F4014491452C440CD3018D916C
:1021A0003D014823642DC8010E94DF09F5014491D7
:1021B000D7018C91482350E024E0559547952A9506
:1021C000E1F761E0640DC8010E94DF095394B8E0B3
:1021D0005B12DFCF98E0E92EF12CE1E0F0E0EC0FAC
:1021E000FD1FEE0DFF1D48EF4E0D208160E0C80180
:1021F0000E948709EFEFEE1AFE0AFEE0EF16F104E7
:1022000061F7E1E0F0E0EC0FFD1FEE0DFF1D42EF86
:102210004E0D208161E0C8010E9487092FEFE21A6C
:10222000F20A34E1E316F10461F75E0145E1A40E20
:10223000B11C50E0B8EF9B2E412C512C320143943D
:10224000E12CF12CD5012C9130E00E2C02C03595FB
:1022500027950A94E2F721703327422F4170652FAA
:102260006E0DE62FF0E0A3E0F595E795AA95E1F76E
:10227000762F9E9E700D1124E00FF11FD301C20135
:1022800004C0880F991FAA1FBB1F7A95D2F7898FA8
:102290009A8FAB8FBC8F232B21F02085898D822BC9
:1022A00004C0898D8095908589238087D8015696B2
:1022B0008D919C915797009769F0DC01ED91FC910D
:1022C0000280F381E02D27965FAF27970995279627
:1022D0005FAD2797BFEFEB1AFB0AE8E0EE16F104BB
:1022E00009F0B0CFFFEFAF1ABF0A585F503109F0C5
:1022F000A7CF60E0C6010E94C30960E0C6010E944A
:10230000FC078FEF93E00E9488278F3711F00C9421
:10231000FA1F67E08091C7019091C8010E94C3092C
:10232000E091C901F091CA01E257FF4F60818091AD
:10233000C7019091C8010E94FC079E012F5F3F4F8B
:10234000388F2F8B8FB7F89440916A0150916B01B1
:1023500060916C0170916D018FBF8091CC01909163
:10236000CD01A091CE01B091CF01342F381B3D8F0C
:10237000830F911DA11DB11D8093CC019093CD01C0
:10238000A093CE01B093CF010091C9011091CA0171
:10239000F0E4FF2E8091C2018F5F8F739091C10195
:1023A000891313C080918001882329F1F80180816D
:1023B000918160918001DC01ED91FC910084F185B7
:1023C000E02D09951092800116C08093C201D801BA
:1023D0008D919C91E091C201F0E0EF57FE4F60813A
:1023E000DC01ED91FC910680F781E02D0995FA94CE
:1023F000F110D0CFD7CF8090C9019090CA0164016D
:10240000B8E0CB0ED11C84010C5F1F4FE12CF12CE6
:10241000ED8DAE2EB12C6E2DF701E658FE4F2081CA
:10242000D6012C93F60133973081822F90E0831BE5
:10243000910997FF03C091958195910905975CF0EB
:10244000D8018C91811107C041E04C9313961C92E6
:102450001E92129713C0D8018C91882379F012969E
:102460008D919C9113978A0D9B1D13969C938E932F
:102470001297803D974010F0D8011C92D8018C91A2
:10248000882379F0231769F02083F40180819181FA
:10249000DC01ED91FC910480F581E02DD6014C9199
:1024A0000995BFEFEB1AFB0AEBE0CE0ED11C055FDE
:1024B0001F4FF6E0EF16F10409F0ADCF6090C901AF
:1024C0007090CA01530128E4A20EB11C8301065B7F
:1024D0001F4F63013FE4C30ED11CE12CF12C4D8D45
:1024E000842E912C5E2CF701EC58FE4F4081D501D3
:1024F0004C934130E9F4F80181819281880D991D56
:10250000928381833497208131818217930780F0F1
:10251000D6018C9181110CC04C93F3018081918183
:10252000DC01ED91FC910280F381E02D6E2D099587
:10253000F80180819681891720F4FD8D8F0FD801D5
:102540008C93F8018081891750F1D5019C912291DB
:10255000921729F1913059F421110EC0D801129629
:102560001C921E921197D6011C9281E006C0911117
:1025700003C081E0213009F080E09083F8011082EF
:10258000882369F0D3018D919C91DC01ED91FC9140
:102590000190F081E02DD5014C91652D0995BFEF9B
:1025A000EB1AFB0AEEE0AE0EB11C025F1F4FFEE01D
:1025B000CF0ED11C26E0E216F10409F093CF409132
:1025C000C9015091CA01FA01EE55FF4F80813D8D3E
:1025D000830F8083C12C8081803120F080518083E3
:1025E000C394F9CFC1101AC0E091C701F091C8019E
:1025F000068517851F706689828993890E94AB09B9
:10260000482F212F30E0B901637077278091C901ED
:102610009091CA01672B09F45AC063C08A0106561B
:102620001F4FDA01A456BF4FBA0168567F4F4A5573
:102630005F4FF8018081882309F43FC0FC90FC0CB7
:10264000FC92FB01B080FD0133972081E1E7FCE0C3
:102650008491822390E034E0959587953A95E1F74F
:10266000A82EE0E7FCE0D490D222FD013197E08073
:10267000E1E7FCE024912E2130E0E4E03595279558
:10268000EA95E1F7E0E7FCE08490B81202C0F216A8
:1026900038F4BD1012C0E820FE1478F0BA1005C05E
:1026A000F21AFC92FB01D08204C0FE18FC92FB01DE
:1026B0008083F8018081815080830B5F1F4F1596C6
:1026C0006B5F7F4FA417B50709F0B3CF8DCF4117CC
:1026D00010F023E001C022E0FC01E356FF4F20830D
:1026E00010C010FD06C04117B0F7FC01E356FF4FC4
:1026F00007C0FC01E356FF4F411710F021E0EFCF78
:1027000010820E945E0F2090C7013090C801D10155
:102710005096ED91FC9151972481C1010696222398
:1027200041F0218532854385622F641B23873487DE
:1027300001C06D8D0E942408F101E684F784A10197
:102740004B575F4FFA01A181B28197010E94062881
:10275000DC01CB01038004C0B695A79597958795BA
:102760000A94D2F7682F6F736783E48120E4E29FB5
:10277000F0011124E60FF11DE05FFE4FE491DA0154
:102780001596EC93159716968C911697882319F049
:10279000E1951596EC93F101EC54FF4F0081118106
:1027A000F8014281442381F1A481B58197010E94FF
:1027B0000628DC01CB01068004C0B695A795979545
:1027C00087950A94D2F7682F6F70608787816817A2
:1027D000D9F020E1429FF0011124E60FF11DE05FE6
:1027E000FA4FF490D8018D919C91DC01ED91FC9110
:1027F0000190F081E02D4F2DD80119966C9109952B
:10280000F801F186808587839101245E3F4F3FAFB9
:102810002EAF6D8DC9010E949A086D8D8101065DF4
:102820001F4FC8010E949A08F101E657FF4F3081FF
:1028300039AFC8010E941B0989ABD1015A960D908E
:10284000BC91A02DBCA7ABA72D913D914D915C9162
:102850002DA73EA74FA758ABF101E45BFF4F1081B6
:10286000112309F484C0DA01C90106E0B695A795E1
:10287000979587950A95D1F749015A01B694A7947F
:1028800097948794881A990AAA0ABB0A329680817B
:1028900081110DC03697A081B0E01196A501940179
:1028A0000E94DC27C72ED82EE92EFF2407C0F10195
:1028B000E75BFF4FC080D180E12CF12CF101EC5A95
:1028C000FF4F80818823E9F03196408151816281F8
:1028D0007381F10126AD89AD0E944D09A82FB0E0AA
:1028E0001196A70196010E94D1276B017C01D101AD
:1028F000DF960C9004C0F694E794D794C7940A949A
:10290000D2F7F101E15BFF4F80818823E9F0319636
:102910004081518162817381F10126AD89A90E94B4
:102920004D09A82FB0E01196A70196010E94D1276A
:102930006B017C01D101DF960C9004C0F694E79402
:10294000D794C7940A94D2F78C149D04AE04BF04A4
:1029500010F475016401B4E1CB16D104E104F10473
:1029600048F4F4E1CF2ED12CE12CF12C03C0C12C82
:10297000D12C76016DA57EA58FA598A90E94692905
:102980009B01AC016BED7FE089E490E40E94872815
:102990004B015C01F101E75AFF4F208131814281F7
:1029A0005381298F3A8F4B8F5C8F3E97608170E007
:1029B00080E090E00E946929F101EC5BFF4F2081EB
:1029C0003181428153810E94D32AF101E05CFF4FA3
:1029D00020813181428153810E9416286F8F78A314
:1029E00089A39AA3C701B6010E9469296B017C01E2
:1029F000812F90E0FC013197EF30F10508F095C58B
:102A0000EC5CFF4F0C94272CA5019401C501B40187
:102A10000E941628A70196010E94D32A4B015C014F
:102A20000E94642B2F8D38A149A15AA10E948728AA
:102A300020E030E040E05FE30E94D32A6B017C019C
:102A4000C501B4010E9482284B015C019B01AC01CD
:102A500060E070E080E89FE30E9415282B013C01B4
:102A600020E030E040E05FE30E94D32AF101E75923
:102A7000FF4F6083718382839383349640825182B7
:102A8000628273823496608371838283938381012F
:102A9000035A1F4F20E030E040E85FE3C701B60172
:102AA0000E941628D8016D937D938D939C93139764
:102AB0000C5F1F4F20E030E040E050ECC501B40156
:102AC0000E94D32AF80160837183828393830C5F11
:102AD0001F4FA7019601D4C0A5019401C501B401FF
:102AE0000E941628A70196010E94D32A4B015C017F
:102AF0000E94642B2F8D38A149A15AA10E948728DA
:102B000020E030E040E05FE30E94D32A6B017C01CB
:102B1000C501B4010E9482284B015C0120E030E035
:102B200040E85FE30E9416282B013C0120E030E0E2
:102B300040E05FE30E94D32AF101E759FF4F608331
:102B4000718382839383349677FA709477F87094C4
:102B50004082518262827382349660837183828361
:102B600093838101035A1F4F20E030E040E85FE388
:102B7000C701B6010E941628F80160837183828321
:102B800093830C5F1F4F20E030E040E050ECC50124
:102B9000B4010E94D32AD8016D937D938D939C93A9
:102BA00013970C5F1F4FA701960160E070E080E86B
:102BB0009FE30E94152848C4A5019401C501B401F2
:102BC0000E941628A70196010E94D32A4B015C019E
:102BD0000E94642B6B017C012F8D38A149A15AA161
:102BE0000E94872820E030E040E05FE30E94D32A83
:102BF0002B013C01C501B4010E9482284B015C01FC
:102C000020E030E040E05FE3C701B6010E94D32A34
:102C1000F101E759FF4F6083718382839383349678
:102C200010821182128213823496DC01CB01B058DB
:102C300080839183A283B3838101035A1F4F20E0D5
:102C400030E040E85FE3C301B2010E941628D801DA
:102C50006D937D938D939C9313970C5F1F4F20E092
:102C600030E040E050ECC501B4010E94D32AF801E5
:102C700060837183828393830C5F1F4FA301920152
:102C800060E070E080E89FE379C3A5019401C5018D
:102C9000B4010E941628A70196010E94D32A4B0175
:102CA0005C010E94642B2F8D38A149A15AA10E947A
:102CB000872820E030E040E05FE30E94D32A6B01E8
:102CC0007C01C501B4010E948228412C512CE0E80E
:102CD0006E2EEFE37E2EF101E759FF4F40825182C5
:102CE0006282738220E030E040E050EC0E94D32A00
:102CF0004B015C01F101E359FF4F608371838283D3
:102D00009383349640825182628273828101035A96
:102D10001F4FA3019201C701B6010E941628F801B6
:102D20006083718382839383349680829182A282AE
:102D3000B382085F1F4FA7019601C301B2011EC3F2
:102D4000A5019401C501B4010E941628A7019601AE
:102D50000E94D32A6B017C010E94642B2F8D38A125
:102D600049A15AA10E94872820E030E040E05FE3BB
:102D70000E94D32A4B015C01C701B6010E94822840
:102D80006B017C01298D3A8D4B8D5C8DC501B401A1
:102D90000E94D32A2B013C01810107591F4F20E0DB
:102DA00030E040E85FE30E941628F80160837183F9
:102DB0008283938320E030E040E050ECC701B6010D
:102DC0000E94D32A6B017C01F101E359FF4F60831C
:102DD000718382839383085F1F4FA301920160E098
:102DE00070E080E89FE30E941528D8016D937D93E1
:102DF0008D939C931397298D3A8D4B8D5C8DC501D6
:102E0000B4010E9487284B015C010451110920E0A4
:102E100030E040E85FE30E941628F8016083718388
:102E2000828393833496C082D182E282F382085FE8
:102E30001F4FA501940124CFA5019401C501B40140
:102E40000E941628A70196010E94D32A4B015C011B
:102E50000E9482282B013C01698D7A8D8B8D9C8D7F
:102E60000E94722B6B017C01C501B4010E94642B8E
:102E70004B015C0120E030E040E85FE3698D7A8D32
:102E80008B8D9C8D0E9415286BA37CA38DA39EA384
:102E9000A30192010E94D32A6DAB7EAB8FAB98AF9A
:102EA00020E030E040E85FE3698D7A8D8B8D9C8D6A
:102EB0000E9416286FA378A789A79AA7A301920159
:102EC0000E94D32A6AAF7BAF8CAF9DAFA70196015A
:102ED000C701B6010E9416286B017C012F8D38A115
:102EE00049A15AA1C501B4010E94872820E030E021
:102EF00040E05FE30E94D32A9B01AC01C701B60109
:102F00000E94D32A2B013C012DA93EA94FA958ADFF
:102F10006FA178A589A59AA50E9415286B017C014F
:102F2000810107591F4FA30192010E9416289B019E
:102F3000AC01698D7A8D8B8D9C8D0E94D32AF8010E
:102F400060837183828393830C5F1F4F298D3A8D39
:102F50004B8D5C8DCA01B9010E9416284B015C01A2
:102F60002AAD3BAD4CAD5DAD6BA17CA18DA19EA109
:102F70000E9415289B01AC01C501B4010E94D32A0F
:102F8000D8016D937D938D939C9313970C5F1F4F86
:102F9000A3019201C701B6010E9415289B01AC0153
:102FA000698D7A8D8B8D9C8D0E94D32AF801608368
:102FB0007183828393832DA93EA94FA958AD6FA138
:102FC00078A589A59AA50E9416286B017C01045159
:102FD0001109A30192010E941628D8016D937D93D7
:102FE0008D939C9313970C5F1F4F2AAD3BAD4CAD57
:102FF0005DAD6BA17CA18DA19EA10E94162820E051
:1030000030E040E050EC0E94D32AE7C0A5019401D3
:10301000C501B4010E941628A70196010E94D32A77
:103020002B013C010E9482284B015C01698D7A8D45
:103030008B8D9C8D0E94722B6B017C01C301B201B0
:103040000E94642B2B013C0120E030E040E85FE36C
:10305000698D7A8D8B8D9C8D0E9415286BA37CA326
:103060008DA39EA3A50194010E94D32A6DAB7EABD4
:103070008FAB98AF20E030E040E85FE3698D7A8D58
:103080008B8D9C8D0E9416286FA378A789A79AA77D
:10309000A50194010E94D32A4B015C01A70196016E
:1030A000C701B6010E9416286B017C012F8D38A143
:1030B00049A15AA1C301B2010E94872820E030E053
:1030C00040E05FE30E94D32A9B01AC01C701B60137
:1030D0000E94D32A2B013C012DA93EA94FA958AD2E
:1030E0006FA178A589A59AA50E9416286B017C017D
:1030F000810107591F4FA30192010E9416289B01CD
:10310000AC01698D7A8D8B8D9C8D0E94D32AF8013C
:1031100060837183828393830C5F1F4F20E030E0D4
:1031200040E050EC698D7A8D8B8D9C8D0E94D32A66
:103130006F8F78A389A39AA3A50194016BA17CA1A9
:103140008DA19EA10E9416289B01AC016F8D78A1D4
:1031500089A19AA10E94D32AD8016D937D938D9362
:103160009C9313970C5F1F4FA3019201C701B601F7
:103170000E9415289B01AC01698D7A8D8B8D9C8DE9
:103180000E94D32AF80160837183828393832DA9DF
:103190003EA94FA958AD6FA178A589A59AA50E940F
:1031A00015286B017C0104511109A30192010E94B1
:1031B0001628D8016D937D938D939C9313970C5F84
:1031C0001F4FA50194016BA17CA18DA19EA10E941E
:1031D00015289B01AC010E941628F80160837183B9
:1031E000828393830C5F1F4FA3019201C5C0A50189
:1031F0009401C701B6010E94D32A0E94B22B4B0151
:103200005C019B01AC010E94D32A6B017C01F1019E
:10321000EF58FF4F60837183828393833897608375
:10322000718382839383810103591F4F9B01AC01FA
:103230000E941628F801608371838283938323EFB1
:1032400034E045EB5FE3C501B4010E94D32A4B0192
:103250005C01005111099B01AC01C701B6010E943C
:10326000162820E030E040E85FE30E941628D801ED
:103270006D937D938D939C9313970C5F1F4F20E06C
:1032800030E040E85FE3C701B6010E9415289B01CA
:10329000AC010E941628F8016083718382839383B6
:1032A0000C5F1F4FA5019401C701B6010E941528AC
:1032B00020E030E040E85FE330C1A5019401C701A0
:1032C000B6010E94D32A0E94B22B4B015C019B01E4
:1032D000AC010E94D32A20E030E040E85FE30E9486
:1032E00016286B017C0180E090E0A0E8BFE3F101CB
:1032F000E759FF4F80839183A283B38338968083FD
:103300009183A283B383349720E030E040E050EC17
:10331000208331834283538323EF34E045EB5FE323
:10332000C501B4010E94D32A4B015C018101035AFB
:103330001F4F9B01AC01C701B6010E941628D8019E
:103340006D937D938D939C9313970C5F1F4F20E09B
:1033500030E040E050E4C701B6010E9415289B010F
:10336000AC010E941628F8016083718382839383E5
:103370000C5F1F4FA5019401C701B6010E941528DB
:10338000CEC0A7019601C501B4010E94D32A0E94B4
:10339000B22B6B017C0120E030E040E450E40E945D
:1033A000D32A4B015C01A70196010E94D32A6B012D
:1033B0007C01F101EF58FF4F608371838283938317
:1033C000389760837183828393839B01AC010E9451
:1033D00016282B013C01F101E359FF4F60837183F3
:1033E000828393838101035A1F4F20E030E040E83D
:1033F0005FE3C501B4010E941628A70196010E944F
:103400001628F80160837183828393830C5F1F4FBA
:1034100020E030E040E050E4C301B2010E941528F2
:10342000D8016D937D938D939C9313970C5F1F4FE1
:10343000A501940160E070E080E89FE30E941528F8
:10344000A70196010E941628F80160837183828388
:1034500093836BC0A7019601C501B4010E94D32AD2
:103460000E94B22B4B015C019B01AC010E94D32A4C
:103470006B017C01F101EF58FF4F20E030E040E4A8
:1034800050E42083318342835383389720833183F0
:1034900042835383349680E090E0A0ECB0EC8083CC
:1034A0009183A283B383C501B4010E94D32A4B0147
:1034B0005C018101035A1F4F9B01AC01C701B6019A
:1034C0000E94162820E030E040E450E40E941628D4
:1034D000D8016D937D938D939C9313970C5F1F4F31
:1034E000A7019601C701B6010E94162820E030E02E
:1034F00040EC50E40E941528F801608371838283B8
:1035000093830C5F1F4FA5019401C701B6010E9470
:10351000152820E030E040E450E40E941628D8014D
:103520006D937D938D939C931397F101E35AFF4F15
:10353000C080D180E280F380810107591F4FA7012D
:103540009601F80160817181828193810E948728B0
:10355000D8016D937D938D939C9313970C5F1F4FB0
:10356000A7019601F80160817181828193810E9497
:103570008728D8016D937D938D939C9313970C5F4F
:103580001F4FA7019601F8016081718182819381AB
:103590000E948728D8016D937D938D939C931397F8
:1035A00000511109A7019601F801608171818281A2
:1035B00093810E948728D8016D937D938D939C936E
:1035C00013970C5F1F4FA7019601F801608171816D
:1035D000828193810E948728D8016D937D938D937A
:1035E0009C931397085D1F4FF8018481958120817A
:1035F00031818217930779F1C184D284C114D10437
:1036000061F043855485DA01ED8DAE0FB11DF801EF
:10361000B487A387CA16DB0618F43583248323C036
:10362000F801E280F380A90160E070E09A01AB014B
:103630002E193F09410951090E94D127960140E006
:1036400050E00E94B2272E0D3F1DD80115963C93E5
:103650002E93149708C0F801228133812817390767
:1036600011F093838283F101EF56FF4FE080F180E8
:10367000BD96F182E0827897F182E0827C96D080DC
:103680004701A12CB12C810106561F4FD801559638
:103690008C9155978823E9F056964D915D916D91E7
:1036A0007C9159971A962C9189AD0E944D09282F2B
:1036B00030E02F5F3F4FD7010E9406284B015C018D
:1036C000F801038404C0B694A794979487940A944D
:1036D000D2F7D80150968C9150978823E9F05196F3
:1036E0004D915D916D917C91549714962C9189A97F
:1036F0000E944D09A82FB0E01196A50194010E94E7
:10370000D1274B015C01F801058004C0B694A79451
:10371000979487940A94D2F7DD20F1F0D801169699
:103720004D915D916D917C9119971A962C918D2DEB
:103730000E944D09A82FB0E01196A50194010E94A6
:10374000D1274B015C01F801038404C0B694A7940F
:10375000979487940A94D2F7D8011F969C928E92E0
:103760001E97AA24BB2453E0880C991CAA1CBB1CDE
:103770005A95D1F72DA53EA54FA558A982169306B7
:10378000A406B50609F440C0ABA5BCA58D929D92D8
:10379000AD92BC92139700E010E060E074E284EF19
:1037A00090E0002E04C0660F771F881F991F0A94AF
:1037B000D2F7A50194010E94E4272F3F310551F073
:1037C00048F081E090E001C0880F0A95EAF7809305
:1037D000020105C00F5F1F4F08301105F1F621509F
:1037E00031093093010120930001B1E0B0936E01E3
:1037F00090910201EBA5FCA58481981728F4809193
:1038000002018483B0936F0180E2898380E290E0BB
:103810000E942D2C9B838A83D10154960D911C917B
:103820005597F80123812223B9F1068117810115EB
:10383000110551F4F101E454FF4F0190F081E02DA6
:1038400080818111A9C06BC02F89388D02171307A1
:1038500089F3009711F00E94C22CD8018C918983C2
:103860008C9190E00E942D2C9B838A8380E099812B
:10387000891700F7282F30E0D8011196ED91FC91BF
:103880001297E20FF31F90814A815B81FA01E20FE8
:10389000F31F90838F5FEBCFF80181818F30C9F4E4
:1038A0008281811116C0F12CD8018C91F81610F686
:1038B0000E946827880F892F881F990B2A813B81D6
:1038C0002115310521F0F901EF0DF11D8083F394ED
:1038D000EBCF20E0D8018C91281708F0ABCF822FD6
:1038E00090E0F8013281E181F0E040E1349FE00DA9
:1038F000F11D112435E0EE0FFF1F3A95E1F7E80FB7
:10390000F91FE05FF94FE4914A815B814115510550
:1039100021F0DA01A80FB91FEC932F5FDBCF918163
:1039200091113AC0F101E45BFF4F8081882309F4D3
:1039300040C11FA21BA200E010E03196FEA7EDA738
:1039400091012B583F4F3A8F298FA10143585F4F68
:103950005E8F4D8FC10187599F4F9EAB8DABD101BB
:10396000A359BF4FBBAFAAAFB4962296FFAFEEAF3D
:1039700022972C5F3F4F38A32F8F4C51510924962B
:103980005FAF4EAF2497049726969FAF8EAF2697D2
:103990005496BCA7ABA7EEC0B9AD2B2FBB0F330B12
:1039A00021583F4F90E00196289FA001299F500D7C
:1039B000389F500D11246281852F0E941B2C43815A
:1039C000682F70E0242F30E0261737070CF0482FBF
:1039D00080E090E0841708F0A5CF2A813B81211573
:1039E000310521F0F901E80FF91F10820196F2CF9D
:1039F000ADA5BEA52C918A819B81222309F4E0C04C
:103A0000009729F0FC01E10FF11DB081BBA3EBA1F0
:103A10006E2FEE0F770B7595679575956795072E49
:103A2000000C880B990B0E946B296B017C01A98DFE
:103A3000BA8D8D909D90AD90BC90AD8DBE8D2D9129
:103A40003D914D915C9129AB3AAB4BAB5CABEDA991
:103A5000FEA920813181428153810E94D32A2B010A
:103A60003C01AAADBBAD2D913D914D915C91C5013D
:103A7000B4010E94D32A9B01AC01C301B2010E9490
:103A800016282B013C01EF8DF8A120813181428164
:103A900053812296AEADBFAD22976D917D918D91F0
:103AA0009C910E94D32A9B01AC01C301B2010E94E8
:103AB00016282B013C012496EEADFFAD2497208102
:103AC00031814281538169A97AA98BA99CA90E945D
:103AD000D32A9B01AC01C301B2010E9415282B011E
:103AE0003C01ABA5BCA52D913D914D915C912696D5
:103AF000EEADFFAD269760817181828193810E9436
:103B0000D32A9B01AC01C301B2010E941528AF8DDD
:103B1000B8A18D929D92AD92BC921397E98DFA8DCA
:103B2000C082D182E282F38229A93AA94BA95CA979
:103B3000ABA5BCA52D933D934D935C931397ED8D51
:103B4000FE8D60837183828393830E943329603862
:103B500071050CF443C06FE78A819B81009721F0C7
:103B6000FC01E10FF11D6083ADA5BEA58C91811113
:103B70003CC01F5F8981181708F43ACFEDA5FEA558
:103B800080818823B1F0602F000F770B880B990B91
:103B90000E946B299B01AC0160E070E080E093E43F
:103BA0000E9487284B015C01E12CF12C8981F816D9
:103BB00048F1F10180A5E754FF4F811163C04CC06B
:103BC000009729F0FC01E10FF11D20812FA33FA1F7
:103BD000632F330F770B880B990B25CF6038FFEFDE
:103BE0007F070CF0B9CF60E8B7CF062E000C770B3B
:103BF00077FF03C071956195710906170CF0B9CF75
:103C0000062FB7CF0A811B810115110521F0F8019C
:103C1000EF0DF11DE0806E2D0E2C000C770B880B44
:103C2000990B0E946B29A50194010E94D32A0E943E
:103C300033296038710534F46038FFEF7F071CF4D6
:103C400060E801C06FE70115110521F0F801EF0DE3
:103C5000F11D6083F394AACF0190F081E02D82855D
:103C6000811109C0A085B18511960D90BC91A02D40
:103C70001C9221E0228740E030E020E0F101EA548C
:103C8000FF4FC1C00190F081E02D8281811103C0FE
:103C90009381992381F390E0019629AD2158289FC3
:103CA000A001299F500D11246481852F0E941B2C97
:103CB0002081682F70E0422F50E0461757070CF420
:103CC000822F811101C081E09091CB01981748F4B7
:103CD000290F281B822FF12C00E010E050E040E07B
:103CE00072C0392F381B832FF6CF2A813B812115D3
:103CF000310521F0D901A40FB11D5C91C52E052E0F
:103D0000000CDD0820853185D90111966D917C91DB
:103D100012976115710529F09B01280F311DD901FA
:103D20001C91212F012E000C330B058002C035950C
:103D300027950A94E2F72C0D3D1D203831050CF42F
:103D400047C02FE76115710521F0DB01A90FB11DF7
:103D50002C932A813B812115310521F0D901A40F33
:103D6000B11D0C91A02F002E000CBB0B6D01078024
:103D700002C0D594C7940A94E2F760857185DB018F
:103D800011966D917C9112976115710521F0680F64
:103D9000711DDB01FC906F2D0F2C000C770B068042
:103DA00002C0759567950A94E2F76C0D21153105EF
:103DB00021F0D901A40FB11D6C9321819F5F922343
:103DC0008F5F82234F5F2981421708F48ECF07C08F
:103DD0002038BFEF3B070CF0B5CF20E8B3CF90936E
:103DE000CB01128648CF6181822F0E941B2C592F54
:103DF0008A819B81552359F0009721F0DC01A20FA5
:103E0000B11D3C932F5F8981281768F318C0009774
:103E100021F0DC01A20FB11D4C913081642F042EE2
:103E2000000C770B032E02C0759567950A94E2F794
:103E3000B62F01C0BB0F3A95EAF73B2FDDCFF1015A
:103E4000E554FF4F408150E0B5E055954795BA9550
:103E5000E1F7E0E020E030E81FE78981281778F5F6
:103E60008A819B81009721F0FC01E20FF11DE08126
:103E70006E2F0E2E000C770B042E02C0660F771FDC
:103E80000A94E2F7603871053CF00097B1F0820FB8
:103E9000911DDC011C9311C06038BFEF7B073CF41F
:103EA000009759F0820F911DDC013C9306C00097EA
:103EB00021F0820F911DDC016C932F5FCECF8EAD70
:103EC0009FAD0E941B094FE750E0B9AD4B1B510954
:103ED000B7FD5395F10120AD30E02F5F3F4F429F7A
:103EE000B001439F700D529F700D1124672F7727EB
:103EF000082E000C990B97FF03C0919581959109AD
:103F0000D101D9964C9150E04F5F5F4F849F900153
:103F1000859F300D949F300D1124220F232F221FD7
:103F2000330B319510E0A0E0EFEFF0E0E61BF70B6C
:103F3000BF0133278981A817F8F48A819B810097F4
:103F400021F0FC01EA0FF11D10811603A001179F5B
:103F5000500D1124452F550F550B249F7001259F9F
:103F6000F00C349FF00C1124009721F08A0F911D62
:103F7000FC01F082AF5FDECFD1015A96ED91FC914A
:103F80005B9780917301811125C090E020917001B1
:103F90008217D0F42A813B812115310521F0D90106
:103FA000A80FB11D9C91A0917101B0917201119661
:103FB0002D913C9112972115310521F0D901A80FBF
:103FC000B11D9C938F5FE2CF809102018483B1E0A9
:103FD000B0936F018A819B81009711F00E94C22CDF
:103FE00080E090E0892B11F40C94A2110E94000053
:103FF0000C94A2118091C7019091C8010E940D0AF2
:104000000C9489118091C00085FFFCCF6093C6009D
:10401000089502970C94022008950895DC011496E7
:10402000ED91FC911597E856FF4F60830895DC01F0
:104030001696ED91FC911797E856FF4F608308950F
:104040000F931F93CF93DF93EC01362F423009F487
:1040500041C028F4442361F0413099F1BBC04430A1
:1040600009F493C008F45AC0453009F498C0B2C0AE
:10407000611102C029AFAEC0DC01AD53BF4F8C91BE
:10408000FE01E80FF11DEB53FF4F90812695269519
:1040900068E1620F861709F49DC06C93FE01EC5332
:1040A000FF4F6083992309F495C0E881F98101905D
:1040B000F081E02D4FE7CE01DF91CF911F910F915D
:1040C0000994611103C0C85BDF4F02C0C55BDF4FBD
:1040D000288380C0622F70E080E090E0311108C03A
:1040E000FE01E15BFF4F20838E01005B1F4F23C069
:1040F000C656DF4F288B0E946929288139814A8161
:104100005B810E94D32A20E030E04FE753E40E9415
:104110008728698B7A8B8B8B9C8B5CC0622F70E0BD
:1041200080E090E031111BC0FE01EC5AFF4F20836C
:104130008E010B5A1F4F0E9469292AAD3BAD4CAD31
:104140005DAD0E94D32A20E030E04FE753E40E94A7
:104150008728F80160837183828393833BC0C656AE
:10416000DF4F2D8B0E9469292E813F81488559851B
:104170000E94D32A20E030E04FE753E40E948728D2
:104180006E8B7F8B888F998F25C0611102C028AFFD
:1041900021C0C454DF4FE881F98120831BC0611125
:1041A00003C0C554DF4F94CFC754DF4FE881F98176
:1041B000228321110FC0838181110CC0828581115E
:1041C00009C0A085B18511960D90BC91A02D1C92BF
:1041D00081E08287DF91CF911F910F91089504971D
:1041E0000C9420206038A1F04034C9F034E0FC0188
:1041F00030A721E021A736AB27AB403881F04F73C1
:10420000FC01EC53FF4F6081640F67FF06C0089507
:10421000403829F0403499F708950C94C807089560
:1042200002970C94F220EF92FF920F931F93CF937B
:10423000DF93EC01162F042F862F90E08930910533
:1042400008F050C1FC01ED5BFF4F0C94272C642F4C
:1042500070E0FB01E05AF34FE491AC89BD891296FE
:10426000EC93FB01E05BF34F64918C899D89DC0149
:1042700011966C93119713962C91222309F432C155
:104280000E94D30B2FC1FE01E45BFF4F4083842FBC
:1042900090E0FC013597E730F105D0F4E45BFF4F87
:1042A000DE01A75ABF4F0C94272C47E25DE16EE96F
:1042B00073E409C049EA5EE963EE7FE304C040E0CD
:1042C00053EF63EB70E44D935D936D937C93139781
:1042D000FE01EB58FF4F1082118212821382349636
:1042E00010821182128213823496108211821282FD
:1042F000138234961082118212821382F3C0842FAB
:1043000090E0FC01E05CF34FE491F0E0EE0FFF1F62
:10431000E05EF34F259134913BA72AA721E02FAB14
:104320009C01205F334FF9014491E42FF0E0EE0F40
:10433000FF1FE05EF34F459154915DA74CA7FC0130
:10434000E050F44F849190E0880F991F8052944F71
:10435000FC01459154915FA74EA7F9012491E22FEA
:10436000F0E0EE0FFF1FE05EF34F8591949199AB63
:1043700088ABB8C0842F90E0FC01E05CF34FE4917F
:10438000F0E0EE0FFF1FE05EF34F259134913D8F7B
:104390002C8F21E029A79C01205F334FF901449124
:1043A000E42FF0E0EE0FFF1FE05EF34F45915491D4
:1043B0005F8F4E8FFC01E050F44F849190E0880FA6
:1043C000991F8052944FFC014591549159A348A3E1
:1043D000F9012491E22FF0E0EE0FFF1FE05EF34FB2
:1043E000859194919BA38AA37DC0FE01E757FF4F5F
:1043F000408378C0DE01AB57BF4F4C93842F90E0D1
:10440000FC01EE0FFF1FE056F44F259134911296F8
:104410003C932E931197FC01E057F44FE4911396CF
:10442000EC9360C0CE0183579F4F9E012A543F4FAB
:104430007901483018F5E0ECFBE025913491DC017E
:1044400018963C932E9317970E946D0E802F880F1D
:10445000F7018283811104C0108281E0818342C010
:10446000982F93709C5FD70190838695869591E0F5
:1044700001C0990F8A95EAF7892F13C0B4E04B9FCA
:10448000F0011124EE55F44F25913491FC01308751
:1044900027830E946D0ED70112961C9212971C92D0
:1044A00081E011968C931EC0FE01EC54FF4FE0801A
:1044B000F180F7014283411115C080819181DC01B7
:1044C000ED91FC910190F081E02D40E8D701199623
:1044D0006C91099580E8F701818704C0642FCE01B3
:1044E0000E94A2078E89181312C0888D998DDC0155
:1044F000ED91FC910190F081E02D20E0402F612FA3
:10450000DF91CF911F910F91FF90EF900994DF9170
:10451000CF911F910F91FF90EF90089504970C9405
:10452000132108958F929F92AF92BF92CF92DF9204
:10453000EF92FF920F931F93CF93DF93CDB7DEB728
:104540002E970FB6F894DEBF0FBECDBF8FE491E07B
:104550009093C4018093C30183E691E09093C601D8
:104560008093C5018091230381113EC18DE191E0CB
:104570009093DE018093DD018FE391E09093E00161
:104580008093DF0185E491E09093E2018093E10163
:104590001092E3011092E4011092E5011092E601FD
:1045A00080E09DE7A0E0B0E08093E7019093E80110
:1045B000A093E901B093EA011092EC011092EB0193
:1045C0001092F3011092F4018FEF9FE79093FA019C
:1045D0008093F9019093FC018093FB019093FE017D
:1045E0008093FD0124E731E0309300022093FF0126
:1045F0001092020210920102109203021092040221
:10460000109205021092060290930802809307020E
:1046100090930A028093090290930C0280930B02FC
:1046200030930E0220930D021092100210920F028E
:1046300010921102109212021092130210921402A0
:10464000109215028FEF80931602E8E1CE2EE2E77A
:10465000DE2EE1EBEE2EEFE3FE2EC0921702D0929B
:104660001802E0921902F0921A0240E440931B02F1
:1046700036E030931C0280E090E0A0E0BFE380933E
:104680001D0290931E02A0931F02B09320028DE999
:104690009CE9ACE9BDE38093210290932202A093B0
:1046A0002302B093240288E78093250280E197E2F9
:1046B00090932702809326021092280221E02093F3
:1046C000290210922A0210922B0210922C021092B0
:1046D0002D0210922E0210922F0210923002109290
:1046E0003102109232021092330210923402109270
:1046F000350280E090E0A0E8BFE380933A02909317
:104700003B02A0933C02B0933D0282E080936202A0
:1047100081E090E0909364028093630284E0809350
:10472000650210926602109267021092680210925F
:10473000690288EB91E090936B0280936A029093F8
:104740006D0280936C0290936F0280936E021092C0
:104750007002109272021092710210927402109202
:1047600073021092760210927502C0927702D09274
:104770007802E0927902F0927A0240937B023093C1
:104780007C0248E152E761E37FE340937D0250936E
:104790007E0260937F027093800240E84093810222
:1047A00057E0509382021092930220939402109249
:1047B00095021092980290939C0280939B02109213
:1047C0009D0210929E0210929F028CE38093A002A1
:1047D0008093A102E2EAF2E0DF011D924A95E9F737
:1047E00030932203209323038DED91E09093C80131
:1047F0008093C7018091CE0381116CC08BE293E05E
:10480000E7E3F3E0AC01DA0113961C921E921297D3
:104810009F0128503109D9011C922F5F3F4FD901C8
:104820001C92DA0117961C921E9216972D5F3F4F2D
:10483000D9011C922F5F3F4FD9011C922F5F3F4F30
:10484000D9011C922F5F3F4FD9011C921082455F06
:104850005F4F3B96B3E04D365B07A9F6EFE6F3E01A
:1048600040ED57E024E11182108253834283DC0142
:10487000A85BBF4F1C9211961C9211961C92108639
:10488000178213961C9211961C9211961C921196E7
:104890002C9311961C923E960E9633E08F37930719
:1048A00011F71092C3031092C4031092C503109223
:1048B000C6031092C7031092C8031092C903109246
:1048C000CA031092CB031092CC031092CD0381E067
:1048D0008093CE038BE293E09093CA018093C90149
:1048E00085EC91E09093F6018093F50188E190E0EA
:1048F0000E942D2C28E0E1E1F1E0DC0101900D9215
:104900002A95E1F7DC0118961C92189719961C92CB
:10491000FC013A962CE0DF011D922A95E9F72FEF72
:10492000FC012287208B21EE31E02115310519F49D
:10493000178A168A02C0378B268B9093F0018093DA
:10494000EF0188E090E00E942D2C8C01FC01118287
:104950001282138260E2F62EF08283E090E00E94E1
:104960002D2C6C01DC01FC9280E290E00E942D2C49
:10497000F60192838183D8011796DC92CE92169726
:1049800080E691E015969C938E93149760E0C801A1
:104990000E94D30B1093F2010093F10185E090E0A7
:1049A0000E942D2C8C0180E097E3A0E0B0E0F8019C
:1049B00080839183A283B3831482F09270018091EB
:1049C000700181508093030183E090E00E942D2CC0
:1049D0006C01DC01FC9280E290E00E942D2CF6013B
:1049E00092838183D092D101C092D00183E090E084
:1049F0000E942D2C6C01DC01FC9280E290E00E9470
:104A00002D2CF60192838183D0927201C0927101A4
:104A10001093F8010093F7018BE090E00E942D2C99
:104A20008C01DC0112961C92129713961C9213971C
:104A300081E015968C93159716968C93169717967A
:104A40008C9317971A961C921A97FC928FE11196E5
:104A50008C93119778E0E72E1496EC9283E090E027
:104A60000E942D2C6C01FC01F08280E290E00E94FB
:104A70002D2CD60112969C938E931197F801D18616
:104A8000C0861093970200939602609122038DEDE9
:104A900091E00E94A2078FE890E00E942D2CFC017B
:104AA0008DE7808311821482158216821782108608
:104AB0001286118614861386158610E89F01225FE0
:104AC0003F4FD901812F1D928A95E9F7DF01A25747
:104AD000BF4F1C928DED91E093838283F093EE01A2
:104AE000E093ED018AE090E00E942D2CFC011282FF
:104AF00082E0838381E090E095838483E68217825D
:104B00008FE0808711878FED91E091838083F09310
:104B10009202E093910284E090E00E942D2CFC012F
:104B200010821182F382E28290939A02809399021A
:104B30000091C9011091CA0183EC91E0D8018D93D5
:104B40009C93F8947801F8013C9680E090E067E847
:104B500080937C0020917C00206420937C00209135
:104B60007C00206220937C0060937A0020917A0080
:104B7000206420937A0020917A0026FDFCCF2091BA
:104B80007900AC0146585E4FDA012C93D701139699
:104B90001C921E921297AF0148505109DA011C92E3
:104BA0004F5F5F4FDA012C93D70117961C921E922C
:104BB00016974D5F5F4FDA012C939F012350310907
:104BC000D9011C922F5F3F4FD9011C922F5F3F4F9D
:104BD000D9011C9210820196BBE0EB0EF11C3B96B2
:104BE0008630910509F0B4CF10927C0080917C0052
:104BF000806480937C0080917C00806280937C0044
:104C00008FE880937A0080917A00806480937A00A4
:104C100052985A9825982D9824982C98209828983E
:104C200057985F9854985C98219A2998239A2B98C2
:104C3000229A2A98559A5D98569A5E98539A5B984C
:104C400083B0D9B0ED2CF12CC7019595879595953A
:104C50008795E82FE1709E2E40ED57E06E2FCE0134
:104C600001960E945C0ED801AC5BBF4F8EE0FE0146
:104C7000319601900D928A95E1F7CE0101960E943E
:104C8000540EF801E05BFF4F89E18083A82CB12C22
:104C9000C50135E0959587953A95E1F7F82FF170C4
:104CA000CF2E40ED57E06F2FCE0101960E945C0E93
:104CB000D801AE5ABF4F8EE0FE01319601900D92A1
:104CC0008A95E1F7CE0101960E94540EC50144E099
:104CD000959587954A95E1F7282F2170A22E40EDF2
:104CE00057E0622FCE0101960E945C0ED801A05AB7
:104CF000BF4F8EE0FE01319601900D928A95E1F74B
:104D0000CE0101960E94540E382D3170832E40ED55
:104D100057E0632FCE0101960E945C0ED801A25984
:104D2000BF4F8EE0FE01319601900D928A95E1F71A
:104D3000CE0101960E94540EDD1CDD24DD1C40EDE9
:104D400057E06D2DCE0101960E945C0ED801A4584B
:104D5000BF4F8EE0FE01319601900D928A95E1F7EA
:104D6000CE0101960E94540EC70154E09595879597
:104D70005A95E1F7A82FA170EA2E40ED57E06A2F6F
:104D8000CE0101960E945C0ED801A657BF4F8EE05F
:104D9000FE01319601900D928A95E1F7CE010196C0
:104DA0000E94540E90927401C0927501A0927601F7
:104DB00080927701D0927801E092790180916B0026
:104DC000806280936B0080916B00806180936B00A8
:104DD00080916B00816080936B00D89A809168000D
:104DE00081608093680080916D00846080936D0085
:104DF00080916D00806880936D0080916D0080616E
:104E000080936D00DA9A80916800846080936800D6
:104E100078942E960FB6F894DEBF0FBECDBFDF910B
:104E2000CF911F910F91FF90EF90DF90CF90BF90A7
:104E3000AF909F908F9008958F929F92AF92BF9264
:104E4000CF92DF92EF92FF92CF93DF93EC016881D4
:104E500079818A819B81611571058105910521F414
:104E600064E279ED8BE597E02DE133EF41E050E02E
:104E70000E94B22749015A019B01AC01A7EAB1E4A3
:104E80000E94D1276B017C01ACEEB4EFA501940127
:104E90000E94DF27DC01CB018C0D9D1DAE1DBF1DC7
:104EA000B7FF03C00197A109B04888839983AA83FB
:104EB000BB839F77DF91CF91FF90EF90DF90CF90F2
:104EC000BF90AF909F908F9008950E941C270895E7
:104ED00087E091E00E941C270895A0E0B0E0809355
:104EE000070190930801A0930901B0930A01089566
:104EF000DC01CB01FC01F999FECF06C0F2BDE1BD9A
:104F0000F89A319600B40D9241505040B8F7089588
:104F1000F999FECF92BD81BDF89A992780B5089581
:104F2000DC01A40FB51F4150504048F0CB01840F65
:104F3000951F2E910E94A12741505040D0F708950F
:104F4000262FF999FECF92BD81BDF89A019700B442
:104F5000021639F01FBA20BD0FB6F894FA9AF99AE2
:104F60000FBE0895052E97FB1EF400940E94C927DA
:104F700057FD07D00E94E42707FC03D04EF40C94A1
:104F8000C92750954095309521953F4F4F4F5F4F22
:104F9000089590958095709561957F4F8F4F9F4FA5
:104FA00008950E940628A59F900DB49F900DA49F80
:104FB000800D911D11240895B7FF0C94D1270E94F4
:104FC000D127821B930B0895A1E21A2EAA1BBB1BAB
:104FD000FD010DC0AA1FBB1FEE1FFF1FA217B307C5
:104FE000E407F50720F0A21BB30BE40BF50B661FDB
:104FF000771F881F991F1A9469F76095709580959F
:1050000090959B01AC01BD01CF010895A29FB00115
:10501000B39FC001A39F700D811D1124911DB29FEC
:10502000700D811D1124911D08955058BB27AA278A
:105030000E942D280C940F2A0E94D62938F00E9435
:10504000DD2920F039F49F3F19F426F40C94AC29A3
:105050000EF4E095E7FB0C94A629E92F0E94342A70
:1050600058F3BA17620773078407950720F079F49D
:10507000A6F50C94562A0EF4E0950B2EBA2FA02D0F
:105080000B01B90190010C01CA01A0011124FF27F5
:10509000591B99F0593F50F4503E68F11A16F040F0
:1050A000A22F232F342F4427585FF3CF46953795EF
:1050B0002795A795F0405395C9F77EF41F16BA0BB4
:1050C000620B730B840BBAF09150A1F0FF0FBB1F62
:1050D000661F771F881FC2F70EC0BA0F621F731FAB
:1050E000841F48F4879577956795B795F7959E3F08
:1050F00008F0B0CF9395880F08F09927EE0F979599
:10510000879508950E94E629E3950C94202A0E9431
:105110009B280C940F2A0E94DD2958F00E94D62962
:1051200040F029F45F3F29F00C94A62951110C940A
:10513000572A0C94AC290E94342A68F39923B1F3BE
:10514000552391F3951B550BBB27AA2762177307AD
:10515000840738F09F5F5F4F220F331F441FAA1F41
:10516000A9F335D00E2E3AF0E0E832D091505040FD
:10517000E695001CCAF72BD0FE2F29D0660F771FAB
:10518000881FBB1F261737074807AB07B0E809F091
:10519000BB0B802DBF01FF2793585F4F3AF09E3F16
:1051A000510578F00C94A6290C94572A5F3FE4F33C
:1051B000983ED4F3869577956795B795F7959F5F59
:1051C000C9F7880F911D9695879597F90895E1E0A5
:1051D000660F771F881FBB1F621773078407BA0704
:1051E00020F0621B730B840BBA0BEE1F88F7E0955F
:1051F000089529F416F00C94A6290C94562A0C94C0
:10520000AC290E943C2AA8F39638A0F707F80F9221
:10521000E8942BE33AEA48EB5FE70E94E92A0F9211
:105220000F920F924DB75EB70F920E949F2AE6EA47
:10523000F0E00E94AF294F915F91EF91FF91E595CA
:10524000EE1FFF1F49F0FE57E0684427EE0F441F92
:10525000FA95E1F74195550B0E94692A0F9007FED8
:105260000C945D2A08950E943A296894B1110C9417
:10527000572A08950E943C2A88F09F5798F0B92F2A
:105280009927B751B0F0E1F0660F771F881F991F7B
:105290001AF0BA95C9F714C0B13091F00E94562A9D
:1052A000B1E008950C94562A672F782F8827B85FAD
:1052B00039F0B93FCCF3869577956795B395D9F7D3
:1052C0003EF490958095709561957F4F8F4F9F4FDD
:1052D0000895E89409C097FB3EF4909580957095E9
:1052E00061957F4F8F4F9F4F9923A9F0F92F96E932
:1052F000BB279395F695879577956795B795F111A7
:10530000F8CFFAF4BB0F11F460FF1BC06F5F7F4F43
:105310008F4F9F4F16C0882311F096E911C0772355
:1053200021F09EE8872F762F05C0662371F096E85E
:10533000862F70E060E02AF09A95660F771F881F2D
:10534000DAF7880F9695879597F9089597F99F67EB
:1053500080E870E060E008959FEF80EC0895DF93AF
:10536000CF931F930F93FF92EF92DF927B018C01FB
:10537000689406C0DA2EEF010E94E62AFE01E89446
:10538000A5912591359145915591A6F3EF010E9484
:105390002D28FE019701A801DA9469F7DF90EF90BC
:1053A000FF900F911F91CF91DF91089500240A94EF
:1053B0001616170618060906089500240A941216F0
:1053C00013061406050608950C94AC290E943C2A85
:1053D000D8F3E894E0E0BB279F57F0F02AED3FE0D8
:1053E00049EC06C0EE0FBB0F661F771F881F28F021
:1053F000B23A62077307840728F0B25A620B730B44
:10540000840BE3959A9572F7803830F49A95BB0F28
:10541000661F771F881FD2F790480C94F42B092E33
:105420000394000C11F4882352F0BB0F40F4BF2BFF
:1054300011F460FF04C06F5F7F4F8F4F9F4F08953F
:10544000EF93E0FF07C0A2EA2AED3FE049EC5FEBF3
:105450000E942D280E940F2A0F90039401FC90585F
:10546000EEECF0E00C94072C57FD9058440F551FBC
:1054700059F05F3F71F04795880F97FB991F61F0D6
:105480009F3F79F087950895121613061406551F4D
:10549000F2CF4695F1DF08C0161617061806991FB9
:1054A000F1CF86957105610508940895E894BB27AE
:1054B00066277727CB0197F908959B01AC0160E03F
:1054C00070E080E89FE30C9487280C94A6290C9444
:1054D000F22B0E943C2AD8F39923C9F3940F511D53
:1054E000A3F39150504094F059F0882332F0660FA6
:1054F000771F881F91505040C1F79E3F51052CF7F0
:10550000880F911D9695879597F908955F3FACF0A8
:10551000983E9CF0BB27869577956795B79508F4DC
:10552000B1609395C1F7BB0F58F711F460FFE8CF56
:105530006F5F7F4F8F4F9F4FE3CF0C94572AFA0135
:10554000DC01AA0FBB1F9B01AC01BF5728F4222727
:1055500033274427507820C0B75190F4AB2F002454
:10556000469537952795011CA395D2F3002071F03D
:10557000220F331F441FB395DAF30ED00C94152875
:1055800061307105A0E88A07B94630F49B01AC018F
:105590006627772788279078309621F020833183FB
:1055A0004283538308950E94E62A0C940F2A0E9496
:1055B000D62938F00E94DD2920F0952311F00C94B3
:1055C000A6290C94AC2911240C94572A0E94342A41
:1055D00070F3959FC1F3950F50E0551F629FF00146
:1055E000729FBB27F00DB11D639FAA27F00DB11D5F
:1055F000AA1F649F6627B00DA11D661F829F2227E8
:10560000B00DA11D621F739FB00DA11D621F839F6E
:10561000A00D611D221F749F3327A00D611D231F44
:10562000849F600D211D822F762F6A2F11249F5792
:1056300050409AF0F1F088234AF0EE0FFF1FBB1F95
:10564000661F771F881F91505040A9F79E3F510554
:1056500080F00C94A6290C94572A5F3FE4F3983EFF
:10566000D4F3869577956795B795F795E7959F5FFE
:10567000C1F7FE2B880F911D9695879597F9089590
:105680000E943C2AE8F09E37E8F09639B8F49E383C
:1056900048F4672F782F8827985FF9CF86957795FC
:1056A000679593959539D0F3B62FB1706B0F711D37
:1056B000811D20F487957795679593950C94D72B4A
:1056C0000C94F22B0C94572A9F930E94E6290F907A
:1056D00007FCEE5F0C94202A19F416F40C94AC2904
:1056E0000C94F22B0E943C2AB8F39923C9F3B6F329
:1056F0009F57550B87FF0E94002C0024A0E640EA2C
:10570000900180585695979528F4805C660F771F16
:10571000881F20F026173707480730F4621B730BE9
:10572000840B202931294A2BA6951794079420250C
:1057300031254A2758F7660F771F881F20F0261754
:105740003707480730F4620B730B840B200D311DB3
:10575000411DA09581F7B901842F9158880F969526
:1057600087950895DF93D92F0E94E629E695D7956E
:105770002AED3FE049E45FE3B33A62077307840729
:105780009507D7953AF0A2EA49EC90680E942D2837
:105790000E940F2AECEEF0E00E94072CDD0F13F0C0
:1057A0000E945D2ADD0F0BF49058DF910895882345
:1057B00071F4772321F09850872B762F07C066234A
:1057C00011F499270DC09051862B70E060E02AF00B
:1057D0009A95660F771F881FDAF7880F9695879539
:1057E00097F908959F3F31F0915020F48795779570
:1057F0006795B795880F911D9695879597F90895A8
:1058000091505040660F771F881FD2F708959F93DD
:105810008F937F936F93FF93EF939B01AC010E9453
:10582000D32AEF91FF910E94AF292F913F914F9181
:105830005F910C94D32A991B79E004C0991F9617A5
:1058400008F0961B881F7A95C9F780950895EE0F8A
:10585000FF1F0590F491E02D0994CF93DF938230E0
:10586000910510F482E090E0E091D803F091D90323
:1058700020E030E0C0E0D0E0309711F1408151816C
:1058800048175907C0F04817590761F4828193817E
:10589000209719F09B838A832BC09093D903809320
:1058A000D80326C02115310519F04217530718F403
:1058B0009A01BE01DF01EF010280F381E02DDCCF10
:1058C0002115310509F1281B390B2430310590F4DD
:1058D00012968D919C9113976115710521F0FB0132
:1058E0009383828304C09093D9038093D803FD01EE
:1058F000329644C0FD01E20FF31F81939193225031
:1059000031092D933C933AC02091D6033091D703AF
:10591000232B41F420910D0130910E013093D703D8
:105920002093D60320910B0130910C0121153105F4
:1059300041F42DB73EB740910F0150911001241B47
:10594000350BE091D603F091D703E217F307A0F4EB
:105950002E1B3F0B2817390778F0AC014E5F5F4FC5
:105960002417350748F04E0F5F1F5093D70340931D
:10597000D6038193919302C0E0E0F0E0CF01DF9184
:10598000CF9108950F931F93CF93DF93009709F45E
:105990008CC0FC013297138212820091D8031091BF
:1059A000D9030115110581F420813181820F931FE4
:1059B0002091D6033091D7032817390779F5F09352
:1059C000D703E093D60371C0D80140E050E0AE1792
:1059D000BF0750F412962D913C911397AD012115FC
:1059E000310509F1D901F3CF9D01DA013383228317
:1059F00060817181860F971F8217930769F4EC010C
:105A000028813981260F371F2E5F3F4F3183208336
:105A10008A819B8193838283452B29F4F093D90358
:105A2000E093D80342C01396FC93EE931297ED01D6
:105A3000499159919E01240F351FE217F30771F424
:105A400080819181840F951F029611969C938E936D
:105A50008281938113969C938E931297E0E0F0E0FD
:105A6000D80112968D919C911397009719F0F80127
:105A70008C01F6CF8D919C9198012E5F3F4F820F44
:105A8000931F2091D6033091D7032817390769F463
:105A9000309729F41092D9031092D80302C01382D0
:105AA00012821093D7030093D603DF91CF911F91F9
:105AB0000F91089581E090E0F8940C945F2D16E02A
:105AC000CAE3D6E004C0FE010E94272C2196CB3306
:085AD000D107C9F7F894FFCFDC
:105AD800700401FF01FFFF010000000000DA0380ED
:105AE80000106000F60008050000000000140DC951
:105AF8000CB00CFA0C69066806670666063E0DAB24
:105B08000C650613212020A107F220FEFF000010DB
:105B180021FCFF00008E22A007EF200000000030CB
:105B28000B9C0A9F096A069F0717200D200220FE7A
:0A5B3800FF00000E200C20092000E1
:00000001FF
